:080000000101000000000000F6
:080008000103010000000000EB
:080010000103030100000000E0
:080018000103030301000000D5
:080020000103030303010000CA
:080028000103030303030100BF
:080030000103030303030301B4
:080038000103030303010100B1
:080040000103010303010000AC
:080048000101000103030100A6
:080050000000000103030100A0
:08005800000000000103030198
:08006000000000000103030190
:0800680000000000000101008E
:08007000000000000000000088
:08007800000000000000000080
:00000001FF
